:060000000200660201830C
:03000B00020240AE
:030013000201CB1C
:10001B0002025353656E64656C61646572205665AC
:10002B007273696F6E20312E302020766F6D203207
:10003B00362E30312E32303031204B6C61757320BF
:10004B004C656964696E67657220496E7465726E82
:10005B00657420446F776E6C6F61647581707590F9
:10006B00FF758C00758A00758911C28CD2B9C28E4E
:10007B00C2BBD288D28AD2B8C2BAC2ACD2A9C2ABE6
:10008B00D2A8D2AAC2B1C2B4C2B5755100D2B7754B
:10009B005200755300755400755500755610755701
:1000AB0000755900755A00755800755B099003323D
:1000BB007A027F00EF93F590317A0FBF08F6DAF2F0
:1000CB00900300D2AFE553255893F590E559B40052
:1000DB000C20B0F1C2B7755901316D80E8E559B408
:1000EB00011830B0E0D2B7755902D2B1316DC2B13F
:1000FB00515C758C00758A00D28CE559B4020E20C8
:10010B00B0C3C28CC2B7755901316D80B8E559B413
:10011B000329C28C515CC2B1C2B4C2B57552007511
:10012B005300755400755500755610755700755969
:10013B0000755A00755800D2B7808A755B0121583B
:10014B00755B022158755B032158755B04C2AFC206
:10015B00B1C2B4C2B5D2B751A220B3FB30B3FD02CA
:10016B0000667E087D007C00DCFEDDFADEF6227D7B
:10017B00007C00DCFEDDFA22C0E0C0D0758C00757F
:10018B008A00755A00D55733D55630755610E55839
:10019B00B4000575582121A67558000555E555B4D1
:1001AB000A197555000554E554B40A0F755400052A
:1001BB0053E553B40A057553000552D0D0D0E03245
:1001CB00C0E0C0D030B3FDE559B400650551E55131
:1001DB00B40405755100E551B40010C2B1C2B4C2EC
:1001EB00B57590D2316D7590CA803AB40110C2B515
:1001FB00C2B4D2B17590A4316D7590CA8027B40288
:10020B0010C2B1C2B5D2B47590D7316D7590CA809A
:10021B0014C2B1C2B4D2B575900112016D7590982C
:10022B00316D7590CA316D7590FF316DD0D0D0E0C6
:10023B0032515C4137C0E0C0D0055AE55AB40A03CD
:10024B00755903D0D0D0E032C0E0C0D0D0D0D0E0D0
:10025B0032C0E07590FF316DE55293F590C2973146
:10026B006D7590FF317AE55393F590316D7590FF75
:10027B00317AE55493F590316D7590FF317AE555F0
:10028B0093F590316D7590C0316D7590CA316D7568
:10029B0090FF316DD0E022C0E07590FF316D75900D
:1002AB00A8316D7590FF317A7590EE316D7590FFB9
:1002BB00317A7590EE316D7590FF317A75908E3184
:1002CB006D7590FF317A7590EE316D7590FF317AC7
:0F02DB00E55B93F590316D7590FF316DD0E022AA
:1003000081D7A494D29888D58090C08AA986A8E87D
:10031000AEC2CAEF97ABCE8EE0EE838FF0EBFEBF9E
:10032000FF01572414521808550010400A290628C6
:0B033000687FBFEFFEF7FDFBFEDF7FE4
:00000001FF
